:0C0000000C9469000C9400000C940000AB
:10000C000C9400000C9400000C9400000C94000064
:10001C000C9400000C9400000C9400000C94000054
:10002C000C9400000C9400000C9400000C94000044
:10003C000C9400000C94CB000C9400000C949800D1
:10004C000C9400000C9400000C9400000C94000024
:10005C000C9400000C9400000C9400001027E80392
:10006C0064000A00010000100001100001000000F3
:10007C0000000A000000000000000000000000006A
:10008C000000000000000000000000000000000064
:10009C000000000000000000000000000000000054
:1000AC0000000A0A0A0A0A0A0A0A0A0A0A0A0A0AB8
:1000BC000A0A020002007A00020004007C0001001F
:1000CC0009037E000000F894EE27EFBBF1E0F5BFCA
:1000DC00E5BF8DE0A2E0BB27ED938A95E9F780E0C0
:1000EC0098E0A0E0B1E0ED930197E9F7EEEBF0E0DA
:1000FC0085919591009761F0A591B591059015901A
:10010C00BF01F00105900D920197E1F7FB01F0CFD3
:10011C00E8E0EEBBEFEFEDBFE8E0EEBFC0E0D3E010
:10012C000C944D03AA93EA93FA93EFB7EA931A93BC
:10013C000A931091C0000091C600E12FEC71E9F414
:10014C00E091CE03EF5FE093CE03E150F0E0EB548F
:10015C00FC4F0083A091CE03A93119F4E0E0E093A9
:10016C00CE03A091D003AF5FA093D003A93129F4A3
:10017C00E0E0E093D003689434F809911991E99187
:10018C00EFBFF991E991A99118950A921A926A9385
:10019C007A938A939A93AA93BA93EA93FA93EFB7C2
:1001AC00EA93E0912B03F0912C033196E0932B030F
:1001BC00F0932C030E946019E1E5F1E00E942822E3
:1001CC000E2E0E946019E3EAF2E00E942822E02938
:1001DC0009F4C3C1A0912903B0912A03E4E1F0E032
:1001EC000E943A220E2EE0910603F0E074970E94D2
:1001FC0065190E942E220E22A0911803EEE00E9497
:10020C001E22E02121F0E0911803EF5F03C025FCD2
:10021C0003C0E0E0E0931803A0911803AE3011F492
:10022C00689425F8E0912903E0930603A091190343
:10023C00A13029F4F79B02C0F79801C0F79AE1E0CE
:10024C002E260E946A190E947319E0939D03F09365
:10025C009E0360939F037093A0030E947A19A1E8F8
:10026C00B3E00E947F190E948619ADEAB3E00E94A8
:10027C007F190E948B190E9494190E945421E093BB
:10028C008103F09382036093830370938403A091A2
:10029C00AD03B091AE038091AF039091B003E0E059
:1002AC00F0E060E772E40E945421E093AD03F09318
:1002BC00AE036093AF037093B0030E9499190E9430
:1002CC009E190E2E0E94A3190E949E19E02161F125
:1002DC00E091AD03F091AE036091AF037091B00368
:1002EC000E948B190E945421E093A903F093AA0356
:1002FC006093AB037093AC030E94A819AFE3B3E017
:10030C000E94B119A091A903B091AA038091AB03EB
:10031C009091AC030E947319E0938903F0938A03C4
:10032C0060938B0370938C030E94B619E0E0F0E0AD
:10033C006AE774E40E94BF190E94C4190E94B62097
:10034C00E0939103F093920360939303709394035F
:10035C000E94CD190E94D2190E94E319A9E5B3E0BD
:10036C000E94E8190E94ED190E94B6190E947C2087
:10037C000E94BF19E093A103F093A2036093A3031F
:10038C007093A403A091B103B091B2038091B30315
:10039C009091B4030E94B620E093B103F093B203A2
:1003AC006093B3037093B4030E94CD19E5E20E94ED
:1003BC00F619ABE5B3E00E94E8190E946A190E9495
:1003CC007223DCF40E94061AA0E0B0E080E89FE300
:1003DC000E945421A091A103B091A2038091A30388
:1003EC009091A4030E940621E0939903F0939A0341
:1003FC0060939B0370939C0309C0E0E0E093990326
:10040C00E0939A03E0939B03E0939C030E940F1AE2
:10041C00AEE1B3E00E944320EC930E94061A0E94C6
:10042C00181A0E94B6200E94211AE0918103F091C3
:10043C00820360918303709184030E942A1A0E94A4
:10044C00992168F5E0918903F0918A0360918B03FF
:10045C0070918C030E942A1A0E94B620E0938503A7
:10046C00F093860360938703709388030E942A1A83
:10047C000E94331A0E94AF20DF01CB010E94A81901
:10048C000E945421A0E0B0E081E695E40E94062190
:10049C00A5E5B3E00E94E819689424F802C0E0E1F5
:1004AC002E260E94061A0E943C1A0E94B620E09347
:1004BC008D03F0938E0360938F03709390030E94CF
:1004CC003C1AE0E0F0E060E87FE30E94992109F03B
:1004DC0008F416C0E0938D03E0938E03E0938F0332
:1004EC00E09390030E94451AEF5FFF4F6F4F7F4FD1
:1004FC000E944E1A0E94451AA9E2B0E00E944723BE
:10050C000E94571AA034E2E4BE07EFE08E07E0E049
:10051C009E0778F0E0E0E0934B03E0934C03E0930C
:10052C004D03E0934E03A9E2B0E00E94601A0E94D2
:10053C0047230E94181A0E9494190E940621ADE2CA
:10054C00B3E00E94B119A0911603AC3308F4F298F1
:10055C00A0911603AC3309F4F29A0E946019A33AE5
:10056C00E2E0BE0709F06AC0A09115030E94651A6B
:10057C000E946A1A0E94601A0E9440220E94731AFA
:10058C00E02191F0E0911603EF5FE0931603E09108
:10059C001503F0E03296A0911603B0E0EA17FB07C2
:1005AC0019F4ECE3E0931603E0E0E0932B03E09303
:1005BC002C03C3940E947A1AE8E5F2E00E943422DC
:1005CC000E2E0E947F1AE021E9F0E0914303F09196
:1005DC0044033196E0934303F09344030E947A1A48
:1005EC000E94841AEA1BFB0BE0934903F0934A0325
:1005FC000E946A1A0E9472232CF4E0E0E0934303F9
:10060C00E0934403ECE3EC15C9F4CC24E091000333
:10061C00EF5FE0930003A0910003AC3379F4E0E0CA
:10062C00E0930003E0910103EF5FE0930103A091DD
:10063C000103A43119F4E0E0E0930103E991EFBF69
:10064C00F991E991B991A9919991899179916991CE
:10065C00199009901895AA93E881E066E0937C00C4
:10066C0085E28A95F1F7E0917A00E064E0937A00F4
:10067C00E0917A00E071E1F3E0917A00E061E093BF
:10068C007A00E0917800F091790021960895EF9727
:10069C0021978EE3A2E0B0E0E0E8F0E00E9487232F
:1006AC00FF2401E020E0E0E8E0936100E0E0E0936B
:1006BC006100EFE0E4B9E1E0E5B9E0E0E7B9E4E0DE
:1006CC00E8B9EAEFEAB9E7EEEBB9E0E0E4BDE3E064
:1006DC00E5BDE0E0E6BDE7BDE8BDE1EAE093800002
:1006EC00E2E0E0938100E0E0E0938500E093840099
:1006FC00E0938700E0938600E0938900E093880004
:10070C00E0938B00E0938A00E093B600E1EAE0937B
:10071C00B000E2E0E093B100E0E0E093B200E093DF
:10072C00B300E093B400E1E0E0936E00E0E0E0930E
:10073C006F00E0937000E0936900EDBBE0936800FC
:10074C00E093C000E8E9E093C100E6E0E093C2006A
:10075C00E0E0E093C500E7E4E093C400E0E8E0BF2C
:10076C00E0E0E0937F00E0937E00E0E6E0937C0025
:10077C00E7E2E0937A00E0E0E0937B00ECBDE093ED
:10078C00BC0078940E94891A0E94911A0E949E1AA9
:10079C000E94AB1AEAE09E1630F4ABE1B0E0E0E068
:1007AC00F0E00E944F23EAE08E1640F4A1E2B0E0A4
:1007BC00E0E0F0E00E944F23689426F8EAE0AE16E1
:1007CC0018F4689430F827F8689433F80E94B51A36
:1007DC000E94BC1A0E94C31AE8ECF0E0E0934F03AD
:1007EC00F0935003EFE0E0930A03A0E0B0E00E9426
:1007FC003B23E0930B03A1E0B0E00E943B23E0938A
:10080C000C03A2E0B0E00E943B23E0930D03A3E0B5
:10081C00B0E00E943B23E0930F03A4E0B0E00E9401
:10082C003B23EE8BA5E0B0E00E943B23EF8BA6E0D0
:10083C00B0E00E943B23E88FA7E0B0E00E943B238E
:10084C00E0931003A8E0B0E00E943B23E093110377
:10085C00A9E0B0E00E943B23E0931203F798F198D3
:10086C00AAE0B0E00E943B23E0931503A9E1B0E0BD
:10087C000E9437230E94CA1AA4E1B0E00E943B23D5
:10088C00EA8BA5E1B0E00E943B23EB8BA6E1B0E044
:10089C000E943B23EC8BABE0B0E00E943B23EE8745
:1008AC00ACE0B0E00E943B23EF87ADE0B0E00E94EB
:1008BC003B23E88BADE1B0E00E943723ED83FE8350
:1008CC00AEE0B0E00E943B23E0931A03AFE0B0E04F
:1008DC000E943B23E0931C03A0E1B0E00E943B2369
:1008EC00E0931B03A9E2B0E00E9433230E944E1A4E
:1008FC00ABE1B0E00E943723ADE7B3E00E94CF1A22
:10090C000E94331AADE2B3E00E94B1190E94181A8A
:10091C000E9494190E9454210E94211AA1E1B0E076
:10092C000E943B233E2FAFE1B0E00E943723E987C2
:10093C00FA87A2E1B0E00E943B23EA8FA3E1B0E08A
:10094C000E943B23E98FA1E2B0E00E943723A1E98A
:10095C00B3E00E94CF1AA3E2B0E00E9437230E94BA
:10096C00D61AA7E2B0E00E9437230E94DB1AA7E157
:10097C00B0E00E943B230E94822323F8A5E2B0E062
:10098C000E9437230E94E01AA8E1B0E00E943B23AA
:10099C00E0930803A0910303A43128F4E09103032E
:1009AC00EF5FE0930303A0910303A431A1F4E0E013
:1009BC00E0932003E0932103EBE0F0E0E0934703A6
:1009CC00F0934803E8EBE0932203E0E0E093CE03DE
:1009DC00EAE0E0930303A091CE03AB30C1F4E091C5
:1009EC00B803E0932003E091B903E0932103E09175
:1009FC00BA03F0E0E0934703F0934803E091BB03A4
:100A0C00E0932203E0E0E093CE03E0930303A09194
:100A1C00CE03AC30C0F0E0E0E093B503E093B60356
:100A2C00E093B703E093B803E093B9030E94B51ABF
:100A3C00E0E0E093BC03E093BD03E093BE03E093DE
:100A4C00BF03E093CE03E8EC5E1630F45394E4E17C
:100A5C00E51511F4E1E04E2E0E94891AA0E00E94E7
:100A6C00E51A3B9798F1A0E00E94EA1A66277727CF
:100A7C000E94F11A0E94ED19A8EEB3E080E090E01C
:100A8C000E948B22DF01CB010E94FA1A662777277E
:100A9C000E94CD220E94F11AE0910903EF5FE093CE
:100AAC000903E0910803A0910903AE1768F00E94B6
:100ABC00ED19E0936D03F0936E0360936F037093E5
:100ACC007003E0E0E0930903E894F3F80E94FF1A46
:100ADC000E94911AA2E00E94EA1ADF01E5E0F0E020
:100AEC000E949022BE2E0E94FF1A0E949E1AA7E01E
:100AFC000E94E51A0E94061B0E94FF1AA5E00E94A4
:100B0C00E51A1E2F0E94FF1AA0E00E94E51ADE2EA5
:100B1C000E94FF1A0E94AB1AE7EAE0937A00A6E063
:100B2C000E94E51AEC87E7E2E0937A00E1E0E51534
:100B3C0091F50E946519E2E3F0E00E943A220E2E34
:100B4C000E940B1B0E943422E02111F0E5E0EB87A0
:100B5C00A12FE2E30E9423220E2EEAEF0E941E2216
:100B6C00E02111F0E6E0EB870E940B1B0E943A2279
:100B7C000E2E0E940F1BE02911F0E7E0EB87A12F4E
:100B8C00EAEF0E9423220E2EEEE10E941E22E029A3
:100B9C0011F0E8E0EB870E940B1B0E943A220E94A6
:100BAC00151B39F0E1E0EB87E8E2F0E00E94061B50
:100BBC0007C00E940F1B0E94151B11F0E2E0EB878F
:100BCC00A12FEAEF0E9423220E94151B11F0E3E0F3
:100BDC0008C0A12FEEE10E941E220E94151B19F0E5
:100BEC00E4E0EB871CE3AB850E94211BAB85E7E0BF
:100BFC000E9405220E2AE1E00E9405220E2AE2E064
:100C0C000E940522E02929F0E12FF0E00E94061B4A
:100C1C0018E2AB850E94261BAB85E8E00E940522FA
:100C2C00E02909F018E20E942B1B0E94311B0E9444
:100C3C001E22E021D1F06894F3F8013021F4F398EE
:100C4C00F49A02E012C0023059F4F498F59AA88D87
:100C5C00A13010F003E003C0F598F39A01E005C051
:100C6C00033019F4F598F39A01E00E946519D397B3
:100C7C0008F457C00E943B1B0E94401BE02F0E94AF
:100C8C00471B20F0E8ECF0E00E94061BE02F0E94CE
:100C9C00571B0E94671BAC91A13008F441C00E9405
:100CAC006E1B0E94771B0E947D234CF40E94671BD5
:100CBC000E94831B0E94C5210E948E1B23C00E9490
:100CCC00971B0E94991BEF930E94971B0E94A21BDB
:100CDC00AF91EA2379F00E94671B0E94831B0E944C
:100CEC00CA21A0935D03B0935E0380935F0390933E
:100CFC00600308C00E94971B0E94AB1B1CF00E9453
:100D0C00B51B0EC0A0915D03B0915E0380915F0393
:100D1C00909160030E94C41B0E94CD220E94061B6E
:100D2C0004C00E94C91B0E94B51B0E94CF1B0E94CD
:100D3C00D51B0E220E94DA1BE02139F0E09127032B
:100D4C00E09317036894F0F821F80E943B1B30974E
:100D5C0021F4E0E0E093180306C0A0911803A23040
:100D6C0010F4E89425F80E943B1BE0932903F093C0
:100D7C002A030E943B1B309719F4E89421F813C006
:100D8C00A0E021FCA1E0E0E00E9405220E2EA09143
:100D9C0017030E94E11B39F0E0E0E09317030E9477
:100DAC00C91BE89422F8A0911703A13040F0689475
:100DBC0022F8E0911703F0E00E94061B02C0E894B1
:100DCC0022F8E09105030E946519F0E0AE17BF0709
:100DDC0020F0E0912703E0930503E0910503F0E098
:100DEC0035970E946519AE17BF0770F4E091270381
:100DFC00E093050325FE08C0E2E0E0931D03E894B0
:100E0C0025F8E0E0E0931803A0911D030E94651AF9
:100E1C000E94E61B0E9450220E22A0911A030E94EF
:100E2C00ED1B1E2EA0911D030E94651A0E94E61B4D
:100E3C000E9448220E22A0911B030E94ED1BE12967
:100E4C0079F00E94C91BA0911D03A13021F4EAE0A6
:100E5C00F0E00E94061BE0911D03E150E0931D039E
:100E6C000E94F21B0E22A0E031FCA1E00E94ED1BBF
:100E7C0031F0689431F80E943B1B0E94081C0E94C0
:100E8C00F21BE02161F10E940D1C0E94151CA4F0C4
:100E9C00A0916903B0916A03ED81FE81EA1BFB0B03
:100EAC00A3E0B0E00E9486220E941D1CAE1BBF0B6B
:100EBC00A0935103B09352030E940D1C0E94722305
:100ECC002CF40E94221C32970E94081CA091520301
:100EDC00AA232AF4E0E0E0935103E09352030E942A
:100EEC00271C0E94782384F5E89431F80E94271C73
:100EFC000E94CA210E94151C74F0AD81BE81E09144
:100F0C006903F0916A03EA1BFB0B0E941D1CEA0F9C
:100F1C00FB1F0E94081C0E94271C0E94CA21A230A1
:100F2C00E0E0BE07E0E08E07E0E09E072CF00E94B8
:100F3C00221C31960E94081C0E941D1CA93CE0E05A
:100F4C00BE0714F00E94BC1A0E94221C0E94651954
:100F5C00EA17FB0720F40E94221C0E94061B0E9429
:100F6C00341C0E94BF210E2EA0E032FCA1E00E9496
:100F7C00ED1B59F0689432F80E946519EAE00E9462
:100F8C008022E0935303F09354030E94341C0E947C
:100F9C00992109F008F435C00E94431CDF01CB01F4
:100FAC00E0E0F0E060E070E40E94992109F008F4C0
:100FBC0010C00E94431CDF01CB01E985FA850E9419
:100FCC00521C0E94591C0E945E1CA3E5B3E00E94B7
:100FDC00E8190E94431C0E94682354F4EA8DF0E047
:100FEC000E94591CAE1BBF0BA0935303B093540328
:100FFC00A0915403AA232AF4E0E0E0935303E09376
:10100C0054030E94341C0E949921F0F5E89432F8A4
:10101C000E94631CDF01CB01E0E0F0E060E470E4CF
:10102C000E94992109F008F418C00E94631CA0E0EA
:10103C00B0E080EA90E40E940621DF01CB01E09150
:10104C005303F09154030E94FB210E947C200E94C8
:10105C00B620A3E5B3E00E94E8190E94631C0E942D
:10106C00682354F4E98DF0E00E94591CEA0FFB1F31
:10107C00E0935303F09354030E94591CA13DE7E005
:10108C00BE0714F00E94C31A0E946519EAE00E9480
:10109C008022DF01E0915303F0915403EA17FB0720
:1010AC0030F40E94591C0E946E1C0E94061B1333C4
:1010BC00A0F0E0E0E0931703E12FF0E0F2970E943C
:1010CC00FB210E947C20A6EFB8E28CE99FE30E94F2
:1010DC0006210E9443201E2F01C010E00E943B1BE2
:1010EC00EB83FC83AB2DE4E60E941E220E2EA0E0C7
:1010FC00F099A1E0E1E00E9405220E94731A0E22F1
:10110C00AA81EDE50E940A22E0211E2E0E94841A7B
:10111C000E947A1A0E9428220E94731C0E947F1A35
:10112C00E021E129E9F0E0912D03F0912E03ABE1F0
:10113C00B0E00E944F230E947B1C0E94D71CE091C0
:10114C000803A8E1B0E00E945723A4E6B0E00E9497
:10115C000C205F98A8EEB3E00E940C200C9453195D
:10116C00E0911103E093B300AA2D0E94361D0E945A
:10117C00D51BE02131F0E894F2F827F8E0E0E09399
:10118C0026030E943B1D0E94D51BE02171F0E091CB
:10119C002603EF5FE0932603A0912603AA3029F4DF
:1011AC00E0E0E0932603E09319030E943B1D0E94AC
:1011BC00481D0E94D51BE02171F06894F2F8E09173
:1011CC001903EF5FE0931903A0911903A33019F4ED
:1011DC00E1E0E0931903E0911903E03029F4E0E039
:1011EC00E093B400F7980FC0A0911903A13019F443
:1011FC00E091120306C0A0911903A23021F4F79AD2
:10120C00EFEFE093B4000E9465190E949E190E2E18
:10121C00A12F0E94E11B01F1E0910403EF5FE09329
:10122C000403A0910403E5E00E9423220E2EE4E1C6
:10123C000E941E22E02141F0E0910403E170AFEF27
:10124C00EA02F001E093B400A0910403A03118F07D
:10125C00E0E0E093040326C0A0E030FCA1E0E1E074
:10126C000E9405220E2EA09119030E94ED1BD1F0B5
:10127C00E0912503EF5FE0932503A0912503A130B6
:10128C0019F4EFEFE093B400A0912503A33019F407
:10129C00E0E0E093B400A0912503A43019F4E0E061
:1012AC00E0932503EAE0E81518F4E894F1F826F841
:1012BC000E94501DA0E026FCA1E00E94561DA0E05B
:1012CC00F1FCA1E00E94561D0E94D51BE02131F0DB
:1012DC006894F1F82F5F283009F420E00E94501D2B
:1012EC00A0911403EFEF0E941E22E02121F0E09167
:1012FC001403EF5F03C0E894F1F8E0E0E09314030B
:10130C00A0911403A431B9F4AA81E0E00E9419223F
:10131C000E2E0E94D51BE02119F0EA81E150EA83E0
:10132C00233610F423E607C020E00E947B1C0E94A9
:10133C00D71CE1E04E2E0E94501DA0E0F1FCA1E074
:10134C000E94561DAA81E4E60E9414220E945B1D95
:10135C0051F06894F1F8EA81EF5FEA83AA81A43630
:10136C0011F4E0E0EA83EAE0E91510F4E894F0F80F
:10137C000E94CF1B0E94DA1B0E22AA81E0E00E9481
:10138C000F220E945B1D51F06894F0F8EA81E15045
:10139C00EA83AA81AF3F11F4E3E6EA830E942B1B98
:1013AC000E94621DC1F00E94681DA9F4A091230344
:1013BC00A43119F4E7E0E0932303E0E0E093240385
:1013CC00E894F3F8A0912303A33028F0E0912303D1
:1013DC00E150E0932303AA2DEAE00E941E220E2E78
:1013EC000E94621DC1F00E94681DA9F4A091230304
:1013FC00A43119F4E7E0E0932303E0E0E093240345
:10140C00E894F2F8A0912303A33028F0E091230391
:10141C00E150E0932303AA2D0E94361DAD2DEAE086
:10142C000E942322E02131F0E0E0E0932403E4E188
:10143C00E0932303EAE0ED1510F4E894F3F80E942E
:10144C002B1B0E94311B0E940522E02109F495C13F
:10145C006894F3F8AA81A13049F4A0910B03A13050
:10146C0028F4E0910B03EF5FE0930B03AA81A23009
:10147C0049F4A0910C03A23328F4E0910C03EB5F28
:10148C00E0930C03AA81A33049F4A0910D03A43678
:10149C0028F4E0910D03EE5FE0930D03AA81A430D4
:1014AC0049F4A0910F03A83228F4E0910F03EF5FE9
:1014BC00E0930F03AA81A53031F4AE89A43618F459
:1014CC00EE89EF5FEE8BAA81A63031F4AF89A4369A
:1014DC0018F4EF89EF5FEF8BAA81A73031F4A88D58
:1014EC00A43618F4E88DEF5FE88FAA81A83049F490
:1014FC00A0911003AF3F28F4E0911003EF5FE0934D
:10150C001003AA81AD3069F4A0912F03B091300380
:10151C00A433E8E0BE0728F40E94FA1A31960E9420
:10152C00CA1AAA81AE3031F4AA89A43618F4EA8911
:10153C00EB5FEA8BAA81AF3031F4AB89A43618F497
:10154C00EB89EB5FEB8BAA81A03131F4AC89A4362B
:10155C0018F4EC89EB5FEC8BAA81A13131F4AE85E8
:10156C00A83C18F4EE85EB5FEE87AA81A23131F42A
:10157C00AF85A83C18F4EF85EB5FEF87AA81A33108
:10158C0031F4A889A83C18F4E889EB5FE88BAA81B0
:10159C00A43169F4A0914103B0914203A835E2E073
:1015AC00BE0728F40E94841A7E960E94E01AAA8133
:1015BC00A53159F4AD81BE81A33AE1E0BE0728F410
:1015CC00ED81FE813196ED83FE83AA81A63149F42B
:1015DC00A0911A03A13028F4E0911A03EF5FE09375
:1015EC001A03AA81A73149F4A0911C03A23328F451
:1015FC00E0911C03EF5FE0931C03AA81A83149F42E
:10160C00A0911B03A13028F4E0911B03EF5FE09342
:10161C001B03AA81A93119F43F3008F43F5FAA815A
:10162C00AA3159F40E94731DAC3BE2E0BE0728F4CA
:10163C000E94781D31960E94D61AAA81AB3159F4BA
:10164C000E94CD19A73EE3E0BE0728F40E947D1D41
:10165C0031960E94DB1AAA81AC3161F4A0E023FC24
:10166C00A1E0A13038F4E0E023FCE1E0EF5F0E9460
:10167C00822323F8AA81AD3169F40E949919AE3DF9
:10168C00E3E0BE0738F40E947A193A96E0933703E8
:10169C00F0933803AA81AE3169F40E94A319A835DE
:1016AC00E2E0BE0738F40E9486193A96E0934503AF
:1016BC00F0934603AA81AF3149F4A0910803AA30F4
:1016CC0028F4E0910803EF5FE0930803AA81AC359E
:1016DC0049F4A0910703AA3F28F4E0910703E65FC1
:1016EC00E0930703AA81AD3531F4AB8DA73018F424
:1016FC00EB8DEF5FEB8FAA81AE3549F4A985BA85E6
:10170C001A9728F4E985FA853196E987FA87AA8130
:10171C00AF3531F4AA8DAA3018F4EA8DEF5FEA8F59
:10172C00AA81A03631F4A98DAA3018F4E98DEF5FA7
:10173C00E98FAA81A13649F4A0911503AC3328F4A2
:10174C00E0911503EF5FE0931503AA81A23649F4EB
:10175C00A0911203AA3F28F4E0911203E65FE093F4
:10176C001203AA81A33649F4A0911103AA3F28F4CD
:10177C00E0911103E65FE0931103EAE0EA1510F43F
:10178C00E894F2F8AA2DEAE00E941E220E2E0E9486
:10179C00481D0E94621D09F492C16894F2F8AA8156
:1017AC00A13049F4A0910B03A13028F0E0910B0378
:1017BC00E150E0930B03AA81A23049F4A0910C03F1
:1017CC00AB3028F0E0910C03E550E0930C03AA81B8
:1017DC00A33049F4A0910D03AD3328F0E0910D0333
:1017EC00E250E0930D03AA81A43049F4A0910F03B9
:1017FC00A53128F0E0910F03E150E0930F03AA818B
:10180C00A53031F4AE89A13018F0EE89E150EE8BA1
:10181C00AA81A63031F4AF89A13018F0EF89E150DC
:10182C00EF8BAA81A73031F4A88DA13018F0E88D88
:10183C00E150E88FAA81A83049F4A0911003A1309F
:10184C0028F0E0911003E150E0931003AA81AD3031
:10185C0069F4A0912F03B0913003AD36E7E0BE07D9
:10186C0028F00E94FA1A31970E94CA1AAA81AE3047
:10187C0031F4AA89A63018F0EA89E550EA8BAA81DE
:10188C00AF3031F4AB89A63018F0EB89E550EB8B17
:10189C00AA81A03131F4AC89A63018F0EC89E5505E
:1018AC00EC8BAA81A13131F4AE85A13018F0EE8514
:1018BC00E550EE87AA81A23131F4AF85A13018F042
:1018CC00EF85E550EF87AA81A33131F4A889A130C7
:1018DC0018F0E889E550E88BAA81A43161F4A09155
:1018EC004103B09142030E946E2328F40E94841A93
:1018FC007E970E94E01AAA81A53159F4AD81BE8170
:10190C00A332E1E0BE0728F0ED81FE813197ED8333
:10191C00FE83AA81A63149F4A0911A03A13028F0C4
:10192C00E0911A03E150E0931A03AA81A73149F41C
:10193C00A0911C03A23028F0E0911C03E150E0932D
:10194C001C03AA81A83149F4A0911B03A13028F0F3
:10195C00E0911B03E150E0931B03AA81A93119F418
:10196C00323008F03150AA81AA3159F40E94731D0B
:10197C00A935E2E0BE0728F00E94781D31970E943D
:10198C00D61AAA81AB3149F40E94CD191B9728F0C5
:10199C000E947D1D31970E94DB1AAA81AC3179F42B
:1019AC00A0E023FCA1E0A13050F0A0E023FCA1E0DA
:1019BC00E1E00E942F23EA1B0E94822323F8AA81D4
:1019CC00AD3161F40E9499190E946E2338F40E9483
:1019DC007A193197E0933703F0933803AA81AE312B
:1019EC0061F40E94A3190E946E2338F40E94861998
:1019FC003197E0934503F0934603AA81AF3149F444
:101A0C00A0910803A23028F0E0910803E150E09384
:101A1C000803AA81AC3539F4A0910703A13018F062
:101A2C00E0E0E0930703AA81AD3531F4AB8DA13032
:101A3C0018F0EB8DE150EB8FAA81AE3551F4A985EE
:101A4C00BA850E946E2328F4E985FA853197E987D7
:101A5C00FA87AA81AF3531F4AA8DA13018F0EA8D3E
:101A6C00E150EA8FAA81A03631F4A98DA13018F08B
:101A7C00E98DE150E98FAA81A13649F4A0911503B3
:101A8C00A13028F0E0911503E150E0931503AA81F1
:101A9C00A23649F4A0911203AB3028F0E091120366
:101AAC00EA50E0931203AA81A33649F4A0911103E2
:101ABC00A13028F0E0911103EA50E093110323FCCC
:101ACC0026C0E0912103A5EAB3E0FF27662777271C
:101ADC000E947C200E941C23A091A503B091A60318
:101AEC008091A7039091A8030E9472233CF40E945A
:101AFC00821D0E948B1D0E94921D09C0E0E0E093A4
:101B0C009503E0939603E0939703E093980323FEE9
:101B1C000CC0AC85B0E00E946E1CA5EAB3E00E943C
:101B2C00CF1A0E94821D0E94921D0E94821DAFE15D
:101B3C00B3E00E944320EC93F0914703E0E0DF0117
:101B4C00E0912203F0E0EA0FFB1FA5E7B3E00E944F
:101B5C007F190E949B1DA0E0B0E080E192E40E94FE
:101B6C0054217F936F93FF93EF930E94731D0E94F8
:101B7C00A41DAF91BF918F919F910E94521CE09335
:101B8C007503F093760360937703709378030E9448
:101B9C00A91DE0E0F0E060E87FE30E94BF210E2E7B
:101BAC000E94A91DE0E0F0E068E472E40E94B92113
:101BBC00E021F9F00E949B1D0E948B1DA5E6B3E06D
:101BCC000E9445200E941C230E949B1DE0937903D8
:101BDC00F0937A0360937B0370937C030E94A91D9E
:101BEC000E9494190E940621A1E3B3E00E94B1194E
:101BFC0015C0E0E0E0936503E0936603E0936703B0
:101C0C00E0936803E0937903E0937A03E0937B031A
:101C1C00E0937C03E0933103E0933203A0919903AA
:101C2C00B0919A0380919B0390919C030E94601A3F
:101C3C000E94BF21EF930E94B21D0E94BF21AF9161
:101C4C00EA23C9F10E94C419E0E0F0E068EC72E408
:101C5C000E9454210E94CD19882799270E94232382
:101C6C000E94E3190E94B41DA0917103B0917203FC
:101C7C008091730390917403E0E0F0E064E172E40E
:101C8C000E940621DF01CB010E940F1A0E945421F1
:101C9C00A0E0B0E080E291E40E9406210E94B41D15
:101CAC00E0917103F091720360917303709174036E
:101CBC00DE010E94E8190E94CF1BA0911303EDEFE7
:101CCC000E941E220E220E94D51BE02129F0E091D9
:101CDC001303EF5FE0931303A92D0E94361DA0910F
:101CEC001303EFEF0E941E220E220E94D51BE0214F
:101CFC0029F0E894F0F8E0E0E0931303A0911303CB
:101D0C00EEE10E9405220E2E0E94D51BE02119F057
:101D1C00E1E0E0931603E0911503E03019F4E0E004
:101D2C00E09316030E946A1A0E94601A0E945022C5
:101D3C000E94731CA09116030E94E11B19F0E1E0B4
:101D4C00E0931603A0911603AC3309F41FEFA09196
:101D5C000703A13028F0E0910703F0E00E94061B76
:101D6C004420C9F4E02FF0E034960E946519AE0FC0
:101D7C00BF1FE12F0E94BD1DA4E00E945619A02F89
:101D8C000E94C71DA09127030E945619A12F0E94E3
:101D9C0056190E94CC1DE1E0E41509F057C044240B
:101DAC00A0910D030E94D51DE0930E03F0E0BC96AC
:101DBC00DF01E0910A03F0E0AE0FBF1FE0910B03CF
:101DCC00F0E0AE0FBF1FE0910C03F0E0AE0FBF1FB1
:101DDC00E0910F03F0E0AE0FBF1FEE89F0E0AE0F05
:101DEC00BF1FEF89F0E0AE0FBF1FE88DF0E0AE0F24
:101DFC00BF1FE09110030E94BD1DACE20E9456195A
:101E0C00A0910A030E945619A0910B030E94561927
:101E1C00A0910C030E945619A0910E030E94561912
:101E2C00A0910F030E945619AE890E945619AF89D2
:101E3C000E945619A88D0E945619A09110030E9459
:101E4C00C71DA0E00E94C71D0E94CC1D233608F0C0
:101E5C0059C3A0E0F799A1E0EA2FE295E07F0E2E9E
:101E6C00A0E0F399A1E0EA2FEE0FEE0F0E0EA0E02A
:101E7C00F499A1E0EA2FEE0FA02DAE0FE0E0F5995A
:101E8C00E1E0EA0FEC8FEAE0E9ABEAABEBABECABF1
:101E9C00EDABEEABEFAB0E94DB1DEAE0EBAFECAFD2
:101EAC00EDAFEEAFEFAF0E94E01DAA34E1E0BE074C
:101EBC00E0E08E07E0E09E071CF4E1E0E093020313
:101ECC000E94E01DE9E4F1E060E070E00E94E91D91
:101EDC00EEE5F1E060E070E00E944822E02119F0AC
:101EEC00E3E0E09302030E94E01DEDE5F1E060E029
:101EFC0070E00E94E91DE8E6F1E060E070E00E940D
:101F0C004822E02119F0E7E0E09302030E94E01D73
:101F1C00E7E6F1E060E070E00E94E91DECE7F1E03B
:101F2C0060E070E00E944822E02119F0EFE0E093BD
:101F3C0002030E94E01DAC37E1E0BE07E0E08E0733
:101F4C00E0E09E071CF0EFE1E09302030E946A1AA6
:101F5C000E94ED1D2CF00E94F51D0E94FB1DEBABA9
:101F6C000E94F51D0E94E722ECABA0911F03AA3042
:101F7C0030F0B0E00E946E1C0E94061EE9AB0E947D
:101F8C000C1EEAAB0E94E01D0E94141E0E94FB1D59
:101F9C00EDAB0E94191E0E94FB1DEEAB0E94191E98
:101FAC000E94E722EFAB203099F50E941F1EE755E7
:101FBC000E94251E0E942F1EA436E0E0BE0720F0D2
:101FCC000E942F1E0E94341E0E942F1E0E94A41DD0
:101FDC000E943F1EEEAF0E942F1E0E94451EEFAFC7
:101FEC00A0910103AA3010F0E2E0E8AFA091010348
:101FFC000E944A1EE9AFA0910003B0E00E946E1C43
:10200C000E94061EEAAFA09100030E944A1EEBAF8D
:10201C00213009F05CC00E94501EE75B0E94251E17
:10202C000E94571AA03AE6E8BE07E1E08E07E0E00E
:10203C009E0748F00E94571AE0EAF6E861E070E06B
:10204C000E94531EEAAF0E94571AA031E7E2BE0766
:10205C00E0E08E07E0E09E0748F00E94571AE0E1AE
:10206C00F7E260E070E00E94531EEBAF0E94571A3B
:10207C00A83EE3E0BE07E0E08E07E0E09E0738F004
:10208C000E94571A0E94C41B0E94531EECAF0E9460
:10209C00571AA436E0E0BE07E0E08E07E0E09E07AA
:1020AC0038F00E94571A0E94141E0E94531EEDAF66
:1020BC000E94571A0E94ED1D28F00E945E1E0E947D
:1020CC00531EEEAF0E945E1E0E94E322EFAF223041
:1020DC0009F06AC00E94501EE75F0E94251EE7E7C8
:1020EC00E9AFE4E7EAAFA0915A03AA2352F4E091D6
:1020FC005903F0915A030E94CF21E0935903F093B6
:10210C005A030E94B21D0E94E319772312F4E0E4F3
:10211C00EEAF0E94B21D0E94E3190E94641E10F4DF
:10212C00E0E4EDAF0E94B21D0E94E3190E946D1E07
:10213C0010F4E0E4ECAF0E94B21D0E94E3190E947F
:10214C00761E10F4E0E4EBAF0E947F1EA031E7E2B4
:10215C00BE072CF00E947F1E0E94841EEBAF0E94D3
:10216C007F1EA83EE3E0BE072CF00E947F1E0E945B
:10217C00891EECAF0E947F1EA436E0E0BE072CF057
:10218C000E947F1E0E948E1EEDAF0E947F1E1A972A
:10219C003CF00E947F1E0E946E1C0E94061EEEAF39
:1021AC000E947F1E0E94931E233009F062C00E9481
:1021BC00501EE7570E94251EEEE3E9AFE4E7EAAFB5
:1021CC00A0915C03AA2352F4E0915B03F0915C03B1
:1021DC000E94CF21E0935B03F0935C030E94991E55
:1021EC00772312F4E0E4EEAF0E94991E0E94641E65
:1021FC0010F4E0E4EDAF0E94991E0E946D1E10F4E5
:10220C00E0E4ECAF0E94991E0E94761E10F4E0E40C
:10221C00EBAF0E949C1EA031E7E2BE072CF00E949F
:10222C009C1E0E94841EEBAF0E949C1EA83EE3E005
:10223C00BE072CF00E949C1E0E94891EECAF0E94CF
:10224C009C1EA436E0E0BE072CF00E949C1E0E944F
:10225C008E1EEDAF0E949C1E1A973CF00E949C1E95
:10226C000E946E1C0E94061EEEAF0E949C1E0E94D5
:10227C00931E243001F50E94501EE7570E94251E24
:10228C00EEE3E9AFE4E7EAAFE0E5EBAFA0911E03C4
:10229C00A43620F0B0E00E948E1EEDAFA0911E037C
:1022AC00B0E00E946E1C0E94061EEEAFA0911E03B1
:1022BC000E944A1EEFAF253041F50E94501EE75791
:1022CC000E94251EE0E0E9AFE5E0EAAFE8E7EBAFFE
:1022DC00A881B981A83EE3E0BE071CF00E94891ECC
:1022EC00ECAFA881B981A436E0E0BE071CF00E94D7
:1022FC008E1EEDAFA881B9810E946E1C0E94061E35
:10230C00EEAFA881B9810E94931E263009F04CC013
:10231C000E94501EE75F0E94251E113030F1ECE048
:10232C00E9AFA12F0E94D51DE436A0E0FA074CF0CE
:10233C00A12FB0E0E8ECF0E00E94A3220E94061E60
:10234C00EAAFA12F0E94D51D3A974CF0A12FB0E017
:10235C00E4E1F0E00E94A3220E94061EEBAFA12F45
:10236C000E94D51D0E94061E1EC0EBE0E9AF0E9424
:10237C00A11EE436A0E0FA0738F0AB81BC81E8EC92
:10238C00F0E00E94A61EEAAF0E94A11E3A9738F018
:10239C00AB81BC81E4E1F0E00E94A61EEBAF0E9491
:1023AC00A11E0E943F1EECAF273009F074C0A09113
:1023BC005503B0915603A135EBEFBE0734F4E1E5BC
:1023CC00FBEFE0935503F0935603A0915503B091A6
:1023DC005603A03BE4E0BE0734F0EFEAF4E0E093F0
:1023EC005503F0935603A0915603AA234AF4E0E454
:1023FC00ECAFE0915503F09156030E94CF2104C03D
:10240C00E0915503F0915603E0935703F093580372
:10241C00A0915703B0915803ECE3F0E00E94A32283
:10242C00E0933B03F0933C030E94A91EECE30E9453
:10243C008022A0915703B0915803AE1BBF0BA09301
:10244C003D03B0933E030E941F1EE75D0E94251EB4
:10245C0024FE1BC00E94A91E1A9710F0E2E0E8AF00
:10246C000E94A91E0E94451EE9AFA0913D03B091A8
:10247C003E030E94A41D0E943F1EEAAFA0913D03A3
:10248C00B0913E030E94451EEBAFE3E7EDAFE8E3EE
:10249C00EEAFE4E5EFAF0E94AE1EAE2FE09120034D
:1024AC000E94B41EEA0F0E94BA1E0E94C31EED8F3A
:1024BC00AB85A130E8F00E94DB1DE9E7EBAFE0E56E
:1024CC00ECAFEDAFAB85B0E00E946E1C0E94061E17
:1024DC00EEAFAB850E944A1EEFAF0E94AE1E0E946B
:1024EC00BA1EE00DED8F0E941F1EE75F0E94251E95
:1024FC00F29B08C00E94AE1E0E94BA1E0E94C31E10
:10250C00EF5FED8F233609F0B3C351E0503130F457
:10251C000E94CC1EEAE0EC935F5FF8CFAA81EBE55A
:10252C000E94D31EEAE50E940522E02911F0EFE19A
:10253C00EA83AA81A03211F4ECE5EA83EA81E03067
:10254C0029F4E0910A03F0E0EF83F887AA81A13027
:10255C0029F4E0910B03F0E0EF83F887AA81A23015
:10256C0029F4E0910C03F0E0EF83F887AA81A33003
:10257C0029F4E0910D03F0E0EF83F887AA81A430F1
:10258C0029F4E0910F03F0E0EF83F887AA81A530DE
:10259C0021F4EE89F0E0EF83F887AA81A63021F4CC
:1025AC00EF89F0E0EF83F887AA81A73021F4E88D5A
:1025BC00F0E0EF83F887AA81A83029F4E0911003AA
:1025CC00F0E0EF83F887AA81A93019F4E0E0EF83FB
:1025DC00E887AA81AA3019F4E0E0EF83E887AA81A2
:1025EC00AB3019F4E0E0EF83E887AA81AC3021F43A
:1025FC00E4E2F0E0EF83F887AA81AD3021F40E9489
:10260C00FA1AEF83F887AA81AE3021F4EA89F0E058
:10261C00EF83F887AA81AF3021F4EB89F0E0EF83E8
:10262C00F887AA81A03121F4EC89F0E0EF83F887D8
:10263C00AA81A13121F4EE85F0E0EF83F887AA811D
:10264C00A23121F4EF85F0E0EF83F887AA81A33162
:10265C0021F4E889F0E0EF83F887AA81A43121F412
:10266C000E94841AEF83F887AA81A53121F4ED81A9
:10267C00FE81EF83F887AA81A63129F4E0911A0331
:10268C00F0E0EF83F887AA81A73129F4E0911C03CD
:10269C00F0E0EF83F887AA81A83129F4E0911B03BD
:1026AC00F0E0EF83F887AA81A93121F4E32FF0E061
:1026BC00EF83F887AA81AA3121F40E94781DEF8359
:1026CC00F887AA81AB3121F40E947D1DEF83F88736
:1026DC00AA81AC3131F4E0E023FCE1E0F0E0EF83DF
:1026EC00F887AA81AD3121F40E947A19EF83F8871B
:1026FC00AA81AE3121F40E948619EF83F887AA8152
:10270C00AF3129F4E0910803F0E0EF83F887AA8158
:10271C00AC3529F4E0910703F0E0EF83F887AA8148
:10272C00AD3521F4EB8DF0E0EF83F887AA81AE355F
:10273C0021F4E985FA85EF83F887AA81AF3521F476
:10274C00EA8DF0E0EF83F887AA81A03621F4E98DB9
:10275C00F0E0EF83F887AA81A13629F4E091150304
:10276C00F0E0EF83F887AA81A23629F4E0911203F6
:10277C00F0E0EF83F887AA81A33629F4E0911103E6
:10278C00F0E0EF83F887AA81E0E00E94D31EE3E03B
:10279C000E94D81EE1E10E94D81EE2E10E94D81EE0
:1027AC00E3E10E94D81EE5E10E94D81EEBE10E94F5
:1027BC00D81EEDE10E940522E02911F0F69A01C025
:1027CC00F698A0E0F699A1E0EA2FE795E0E0E7950E
:1027DC00EE8FE0E0ED8FEC8FE0930203AA81B0E086
:1027EC00A7FDBFEF0E946E1C0E94061EEBABAA81D8
:1027FC00B0E0A7FDBFEFEAE0F0E00E94D522ECAB21
:10280C00AF81B885A031E7E2BE0728F0E0E1F7E23E
:10281C000E94A61EEBAFAF81B885A83EE3E0BE07D1
:10282C0028F0E8EEF3E00E94A61EECAFAF81B8856D
:10283C00A436E0E0BE0710F00E94341EAF81B885CC
:10284C001A9728F00E94DD1E0E943F1EEEAFAF814A
:10285C00B8850E94451EEFAFEA81E03061F4EDE6E9
:10286C00EDABE9E7EEABE8E7EFABEDE6EAAFE4E5BD
:10287C00EBAFE0E5ECAFAA81E1E10E94D31EE2E10F
:10288C000E94D81EE3E10E94D81EE5E10E94D81EEA
:10289C00EDE10E940522E02929F00E94DD1E0E9434
:1028AC003F1EEEAFE7EAE0937A00A7E00E94E51A3C
:1028BC000E94061BE7E2E0937A00AA810E94211B8A
:1028CC00AA81EEE00E94D81EE1E10E940522E029D7
:1028DC0011F0E1E06E2EAA810E94261BAA81EFE086
:1028EC000E94D81EE2E10E940522E02911F0E2E0EC
:1028FC006E2EAA81E7E00E94D31EE0E10E94D81E52
:10290C000E94E01E11F0E3E06E2E0E946519D39731
:10291C0008F457C00E943B1B0E94401BE62D0E94EE
:10292C00471B20F0E8ECF0E00E94061BE62D0E940D
:10293C00571B0E94E51EAC91A13008F441C00E94C7
:10294C00EC1E0E94771B0E947D234CF40E94E51E16
:10295C000E94F51E0E94C5210E94001F23C00E94E8
:10296C00091F0E94991BEF930E94091F0E94A21B32
:10297C00AF91EA2379F00E94E51E0E94F51E0E9499
:10298C00CA21A0936103B093620380936303909375
:10299C00640308C00E94091F0E94AB1B1CF00E941C
:1029AC000B1F0EC0A0916103B09162038091630371
:1029BC00909164030E94C41B0E94CD220E94061BAE
:1029CC0004C00E94C91B0E940B1FAA81AD3061F488
:1029DC000E94131F0E94141E0E94FB1D0E941C1FAC
:1029EC000E94231FE0E2EC8FAA81A53161F40E94C2
:1029FC00131F0E94141E0E94FB1D0E941C1F0E948C
:102A0C00231FE0E6EC8FAA810E94211BAA81EEE035
:102A1C000E94D81EE1E10E940522E029A9F00E9443
:102A2C002D1FE4E00E94311F18F00E94371FEDAB00
:102A3C000E9465191A9728F00E943B1F0E943F1EA6
:102A4C00EEAB0E943D1FEFABAA810E94261BAA8110
:102A5C00EFE00E94D81EE2E10E940522E029A9F0D5
:102A6C000E942D1FE2E00E94311F18F00E94371FB8
:102A7C00EDAB0E9465191A9728F00E943B1F0E942B
:102A8C003F1EEEAB0E943D1FEFABAA81E7E00E9418
:102A9C00D31EE0E10E94D81E0E94E01EA9F00E9405
:102AAC002D1FE1E00E94311F18F00E94371FEDAB83
:102ABC000E9465191A9728F00E943B1F0E943F1E26
:102ACC00EEAB0E943D1FEFABAA81A43199F40E949A
:102ADC003F1FE4E6F0E00E94A61EEDAB0E943F1FF4
:102AEC000E94A41D0E943F1EEEAB0E943F1F0E943D
:102AFC00451EEFABAA81A63121F40E94441FEBE0E6
:102B0C00ECAFAA81A73121F40E94441FE0E4ECAFA2
:102B1C00AA81A83121F40E94441FECE0ECAFAA81F9
:102B2C00A93169F4A0911F03B0E00E946E1C0E94B1
:102B3C00061EEDAB0E940C1EEEABE7E7EFABAA81D5
:102B4C00AA3199F40E944B1FE4E6F0E00E94A61E05
:102B5C00EDAB0E944B1F0E94A41D0E943F1EEEABCA
:102B6C000E944B1F0E94451EEFABAA81AB3159F45A
:102B7C00ECE7E9AFE7E7EAAFE8E7EBAF0E94DD1E71
:102B8C000E943F1EEEAFAA81EDE10E94D31EEEE142
:102B9C000E940522E029D9F0E3E7E9AFE8E3EAAFC8
:102BAC00AA81AD3111F4EEE501C0E8E7EBAF0E946C
:102BBC00501F1A9738F00E94501F0E94A41D0E94AB
:102BCC003F1EEEAB0E94501F0E94451EEFABAA8128
:102BDC00E1E10E94D31EE2E10E94D81E0E94E01E99
:102BEC0011F0E8E7EAAFAA81AD3541F5E7E7ECAFC4
:102BFC00EEE5EDAFE9E3EEAFEB8DEFAFE7EAE09397
:102C0C007A00AB8D0E94E51A7E2EE7E2E0937A0003
:102C1C00E3E6E71528F4A72DB0E00E948E1EEDAB7D
:102C2C00E9E0E71538F4A72DB0E00E946E1C0E9475
:102C3C00061EEEABA72D0E944A1EEFABAA81AE3545
:102C4C0021F4EEE5E9AFE1E0EAAFAA81AF3521F47A
:102C5C00EEE5E9AFE2E0EAAFAA81A03621F4EEE5B9
:102C6C00E9AFE3E0EAAFAA81A23611F4E0E1EC8F20
:102C7C0051E0503108F077C00E94CC1EEC91E0304E
:102C8C0021F40E94CC1EEFE3EC930E94CC1EAC917D
:102C9C00A63021F40E94CC1EEDE7EC930E94CC1ED2
:102CAC00AC91A13021F40E94CC1EE6E0EC930E9482
:102CBC00CC1EAC91A23021F40E94CC1EEBE5EC931F
:102CCC000E94CC1EAC91A33021F40E94CC1EEFE4E8
:102CDC00EC930E94CC1EAC91A43021F40E94CC1E2B
:102CEC00E6E6EC930E94CC1EAC91A53021F40E9438
:102CFC00CC1EEDE6EC930E94CC1EAC91A73021F4D7
:102D0C000E94CC1EE7E0EC930E94CC1EAC91A83044
:102D1C0021F40E94CC1EEFE7EC930E94CC1EAC91E8
:102D2C00A93021F40E94CC1EEFE6EC930E94CC1E3D
:102D3C00AC91AA3021F40E94CC1EE0E0EC930E94EE
:102D4C00CC1EAC91AB3021F40E94CC1EE1E0EC9394
:102D5C000E94CC1EAC91AC3021F40E94CC1EE8E059
:102D6C00EC935F5F86CFE0910203E695E6950E94B7
:102D7C00551FEDA90E945B1FEDA90E94661FEDA9CE
:102D8C000E94711FEDA90E94781FEDA90E947F1F60
:102D9C00EDA90E94861FEDA90E948D1FE8A3E0916A
:102DAC000203E695E695E6950E94551FEEA90E9452
:102DBC005B1FEEA90E94661FEEA90E94711FEFA96E
:102DCC000E94781FEFA90E947F1FEFA90E94861F07
:102DDC00EFA90E948D1FE9A3E0910203E6950E94E2
:102DEC00551FEFA90E945B1FEFA90E94661FEFA958
:102DFC000E94711FEEA90E94781FEEA90E947F1FEE
:102E0C00EEA90E94861FEEA90E948D1FEAA3E8ADD1
:102E1C000E94551FE9AD0E945B1FE9AD0E94661F21
:102E2C00E9AD0E94711FEE8D0E94781FEE8D0E94FD
:102E3C007F1FEE8D0E94861FE0910203E170EA2B4A
:102E4C00EBA3EDAD0E94551FEDAD0E94931FEDADB0
:102E5C000E949C1FEDAD0E94A51F0E94AF1FEDADFF
:102E6C000E94B31FEDAD0E94BC1FEDADE295E17069
:102E7C00EA2BECA3ECAD0E94551FECAD0E94931F06
:102E8C00ECAD0E949C1FECAD0E94A51FE2950E9428
:102E9C00781FEEAD0E94B31FEEAD0E94BC1FEEADCD
:102EAC00E295E170EA2BEDA3EE8D0E94C51FECAD0F
:102EBC000E945B1FECAD0E94661FECAD0E94711F5F
:102ECC00EBAD0E94781FEBAD0E947F1FEBAD0E9413
:102EDC00861FEBAD0E948D1FEEA3EEAD0E94551F19
:102EEC00EEAD0E94931FEEAD0E949C1FEEAD0E94B2
:102EFC00A51F0E94C91F0E94781FEBAD0E94B31F33
:102F0C00EBAD0E94BC1FEBADE295E170EA2BEFA399
:102F1C00EAAD0E94551FEAAD0E94931FEAAD0E94D4
:102F2C009C1FEAAD0E94A51FEE1FE0E0EE1F0E9461
:102F3C00781FEFAD0E94B31FEFAD0E94BC1FEFAD29
:102F4C00E295E170EA2BE8A7ED8DE2950E94551F02
:102F5C00EAAD0E945B1FEAAD0E94661FEAAD0E94BB
:102F6C00711FE9AD0E94781FE9AD0E947F1FE9AD8A
:102F7C000E94861FE9AD0E948D1FE9A7EFAD0E944C
:102F8C00551FEFAD0E94931FEFAD0E949C1FEFAD3C
:102F9C00E695E695E6950E94CE1FE9A9EE1FE0E0C6
:102FAC00EE1F0E94781FE9A9E295E170EE0FEE0F7B
:102FBC00EA2BAE2FE9A90E94BC1FE9A9E295EF709C
:102FCC00E695E170EA2BEAA7E9A9E695E695E69580
:102FDC000E94551FE9A9E695E6950E94D41FE9A920
:102FEC000E94DC1FE9A90E94CE1FED8D0E94AF1F2D
:102FFC00ED8D0E94B41EEA2BAE2FED8D0E94E41FC6
:10300C00ED8DE695E170EA2BEBA7ED8D0E94C51FC7
:10301C00EAA9E2950E94D41FEAA90E94661FEAA9B8
:10302C000E94E91FEAA90E94AF1FEAA90E94B41EE0
:10303C00EA2BAE2FEAA9E6950E94E41FEAA9E170FB
:10304C00EA2BECA7ED8D0E94C91F0E94551FEC8D39
:10305C000E94D41FEC8D0E94DC1FEC8DE695E6954A
:10306C000E94CE1FE0910203E2950E94781FED8D25
:10307C00EE1FE0E0EE1FE170EE0FEE0FEA2BAE2F2D
:10308C00EC8DE695E695E6950E94E41FEC8DE295B5
:10309C00E170EA2BEDA7EC8D0E94C51FEBA9E29520
:1030AC000E94D41FEBA90E94661FEBA90E94E91F86
:1030BC00ECA90E94AF1FECA90E94B41EEA2BAE2F04
:1030CC00ECA9E6950E94E41FECA9E170EA2BEEA7AF
:1030DC00EC8D0E94C91F0E94551FECA9E2950E941D
:1030EC00D41FECA90E94661FECA90E94E91FEBA952
:1030FC000E94AF1FEBA90E94B41EEA2BAE2FEBA9C6
:10310C00E6950E94E41FEBA9E170EA2BEFA733FED2
:10311C000DC051E0513150F4E52FF0E0DE015F9627
:10312C00AE0FBF1FEFEFEC935F5FF4CF0E94ED1F6C
:10313C005D3078F40E94F31FA2E5B8E00E94E32111
:10314C00E17011F45D9801C05D9A0E94FA1F5F5FF7
:10315C00EFCF0E9402205D3078F40E94F31FA0E3B1
:10316C00B8E00E94E321E17011F45D9801C05D9A12
:10317C000E94FA1F5F5FEFCF0E9402205D3078F44F
:10318C000E94F31FA2E0B8E00E94E321E17011F469
:10319C005D9801C05D9A0E94FA1F5F5FEFCF0E949D
:1031AC0002205D3078F40E94F31FA6E0B8E00E9484
:1031BC00E321E17011F45D9801C05D9A0E94FA1F41
:1031CC005F5FEFCF0E9402205A3098F45E9885E240
:1031DC008A95F1F7E9E0E51BA0E4B1E00E94E32158
:1031EC00E17011F45D9801C05D9A0E94FA1F5F5F57
:1031FC00EBCF41E04131E8F451E05930C0F45E9836
:10320C0085E28A95F1F7E42FF0E0DE015F96AE0FD0
:10321C00BF1FAC91E8E0E51B0E94DB21E17011F4CB
:10322C005D9801C05D9A0E94FA1F5F5FE6CF4F5F09
:10323C00E1CF5D9A85E28A95F1F7289A8DEC9AE0B8
:10324C000197F1F70E94CF1BA82DEAE00E941E22E5
:10325C000E2AAA2DEAE00E941E220E2AAD2DEAE0CB
:10326C000E941E22E02929F0E0E0E0934303E09362
:10327C004403AB2DE4E60E9423220E2EA0E0F0992D
:10328C00A1E00E94ED1B39F0A4E6B0E00E940C20F6
:10329C00F09AE89433F80C94D004EF962196FFCF73
:1032AC00AA93E091C000E072E1F3E881E093C600DC
:1032BC0021960895A0912B03B0912C030895A09111
:1032CC002703B09128030895A0917903B0917A0354
:1032DC0080917B0390917C030895E0E0F0E061EE37
:1032EC0075E40E9454210895E0913703F09138035E
:1032FC000895662777270E947C200E941C2308953E
:10330C00E0914503F09146030895A0918103B0919B
:10331C00820380918303909184030895E0E0F0E0B0
:10332C0060E271E40895A0913703B09138030895D9
:10333C00E0E0F0E00E943A220895A0914503B0919C
:10334C0046030895E091A903F091AA036091AB03A1
:10335C007091AC0308950E944320ED93FC93089563
:10336C00A0919503B0919603809197039091980347
:10337C0008950E940621DF01CB01AFCFA0919103EC
:10338C00B091920380919303909194030895A0912E
:10339C003903B0913A030895E4E60E948022DF01DC
:1033AC00E0919103F09192036091930370919403D7
:1033BC00882799270E94232308950E9426230E9480
:1033CC00AF2008950E944520ED93FC930895E09161
:1033DC006903F0916A0360916B0370916C0308951B
:1033EC000E948022DF01E091B103F091B203609161
:1033FC00B3037091B403882799270E942323DDCF50
:10340C00E0919D03F0919E0360919F037091A00346
:10341C000895E0919903F0919A0360919B03709148
:10342C009C030895A0917D03B0917E0380917F034E
:10343C00909180030895E0937D03F0937E03609355
:10344C007F03709380030895A0918503B091860348
:10345C0080918703909188030895E0917D03F0910A
:10346C007E0360917F03709180030895A0918D037A
:10347C00B0918E0380918F03909190030895E09109
:10348C004B03F0914C0360914D0370914E030895E2
:10349C00E0934B03F0934C0360934D0370934E03F6
:1034AC000895A0914B03B0914C0380914D039091E2
:1034BC004E030895E0E0F0E060E070E00895E0E095
:1034CC000E9423220E2E0895A0916503B0916603ED
:1034DC00809167039091680308950E22A0911603C2
:1034EC00ECE30E941E220895A0914303B091440383
:1034FC000895A0914103B09142031ACFE09141038A
:10350C00F09142030895A4E1B0E00E940C20E7EA98
:10351C00E0937A000895A4E00E943103EF2FF0E0CD
:10352C009E2EE7E2E0937A00E7EAE0937A000895B2
:10353C00A3E00E943103EF2FF0E08E2EE7E2E09340
:10354C007A00E7EAE0937A000895A1E00E94310343
:10355C00EF2FF0E0AE2EE7E2E0937A000895EBE077
:10356C00E093BA03E8EBE093BB030895E8ECF0E0DA
:10357C00E0935103F09352030895E0EDF7E0E093EC
:10358C005303F09354030895E0932F03F093300307
:10359C0008950E94FB210E947C200E941C23089508
:1035AC00E0933503F09336030895E0933903F093D9
:1035BC003A030895E0934103F093420308950E9467
:1035CC003103EF2FF0E008950E9431030E94F021A7
:1035DC000E94EC210895E0936903F0936A036093D1
:1035EC006B0370936C030895E0912F03F0913003FB
:1035FC000895E7E2E0937A00E7EAE0937A00089511
:10360C00E0932703F0932803089559DEEAEFF0E0E6
:10361C00089555DEEEE1F0E00E94342208950E2E5E
:10362C00A52DE1E00E9423220E22AB85E5E00E944D
:10363C001E22E0210895E5E00E9405220E2E089539
:10364C00E6E00E9405220E2E0895AD2DEAE00E94C0
:10365C001E220E2E0895A0E0F3FCA1E0E0E00E94F3
:10366C0005220E22A22FE3E60895E0912703F091A4
:10367C0028030895F297ADE7B0E00E9458220F019D
:10368C000895F0E0DE015196AE0FBF1FEC91F0E013
:10369C00D0010E949022B4DF12DEA93CE0E0BE070C
:1036AC000895F0E0DE015596AE0FBF1FEC91F0E0EF
:1036BC0006DE0E945822DF01E4E6F0E00E94902230
:1036CC009FCFE02FF0E0DE011D96AE0FBF1F0895D7
:1036DC00A0915D03B0915E0380915F0390916003B4
:1036EC000895E8EEF3E060E070E00E94CD22DF0187
:1036FC00CB01BBDF662777270895EC91F0E00E94A1
:10370C00FB21A8E0BCE481E090E00E94CD22E0CF58
:10371C00E0935D03F0935E0360935F03709360032B
:10372C000895D6DFDECF0E94CA21E5E0F0E060E02C
:10373C0070E00E94502208950E94CA21E4E1F0E05A
:10374C0060E070E00E94482208950E94CA21A431D2
:10375C00E0E0BE07E0E08E07E0E09E070895E09110
:10376C006503F09166036091670370916803A0E5AF
:10377C00B4E180E090E00E948B22CACFE8EEF3E047
:10378C0060E070E00895E0E0E0932703E093280305
:10379C000895A92DEAE00E941E220E2E0895A22F54
:1037AC00E3E60E941E220895A0E0F0FCA1E0E0E018
:1037BC000E9405220895E0E00E942322E021089552
:1037CC00E0911C0381DEFF27662777270895E0E050
:1037DC000E940522E0210895ED81FE81A0916903EC
:1037EC00B0916A0380916B0390916C0366277727E5
:1037FC000E9448220E2EEAE0F0E060E070E00E94A9
:10380C0050220895E0935103F09352030895DFDDA5
:10381C00AD81BE81882799270E94CA210895A630C0
:10382C00E0E0BE07E0E08E07E0E09E070895A0917F
:10383C005103B09152030895E0915103F09152035A
:10384C000895ED81FE81A0916903B0916A03809186
:10385C006B0390916C03662777270895E32FA09153
:10386C00A503B091A6038091A7039091A803FF270D
:10387C00662777270E947C200895E32FF0E0A09123
:10388C00A503B091A6038091A7039091A8030E9471
:10389C00FB210E947C2091CD662777270E947C20FB
:1038AC000E9406210895A0915303B09154030895EA
:1038BC000E9400220E94232380CDA32FBB27E091DE
:1038CC00A503F091A6036091A7037091A803F0CF14
:1038DC00EAE0F0E00E94A32208950E2EA0911603B8
:1038EC00ECE30E941E220E220895E0910B03A0E04F
:1038FC00B0E00E945723E0910C03A1E0B0E00E94DD
:10390C005723E0910D03A2E0B0E00E945723E09111
:10391C000F03A3E0B0E00E945723EE89A4E0B0E0CF
:10392C000E945723EF89A5E0B0E00E945723E88D51
:10393C00A6E0B0E00E945723E0911003A7E0B0E0AE
:10394C000E945723E0911103A8E0B0E00E94572396
:10395C00E0911203A9E0B0E00E945723E091150317
:10396C00AAE0B0E00E9457233FDEA9E1B0E00E943C
:10397C004F23EA89A4E1B0E00E945723EB89A5E12B
:10398C00B0E00E945723EC89A6E1B0E00E945723D7
:10399C00EE85ABE0B0E00E945723EF85ACE0B0E0E1
:1039AC0008950E945723E889ADE0B0E00E945723A8
:1039BC00ED81FE81ADE1B0E00E944F23E0911A034E
:1039CC00AEE0B0E00E945723E0911C03AFE0B0E002
:1039DC000E945723E0911B03A0E1B0E00E94572303
:1039EC00E32FA1E1B0E00E945723E985FA85AFE10E
:1039FC00B0E00E944F23EA8DA2E1B0E00E94572371
:103A0C00E98DA3E1B0E00E945723E0919103F0917E
:103A1C0092036091930370919403A1E2B0E00E9431
:103A2C0045200E944F23E0913503F0913603A3E229
:103A3C00B0E00E944F23E0913903F0913A03A7E2E2
:103A4C00B0E00E944F23E0E023FCE1E0A7E1B0E00E
:103A5C000E94572353DDA5E2B0E00E944F23089546
:103A6C00EAE00E9423220E2E0895AA2DEAE00E947D
:103A7C001E220E2EA0E027FCA1E0E0E00E94052211
:103A8C000E220895A0E0F2FCA1E0E0E00E940522E5
:103A9C000E220895A82DEAE00E941E220E2E0895F3
:103AAC00E0E00E9405220E2208950E22A22FE3E6EA
:103ABC000E940522E0210895A22FE3E60E94052230
:103ACC00E0210895E0912403EF5FE0932403E0915B
:103ADC002303A0912403EA170895A0913503B09114
:103AEC0036030895E0913503F09136030895E09183
:103AFC003903F0913A030895E091A503F091A603E0
:103B0C006091A7037091A8030895A0E0B0E080E055
:103B1C009FE30E94B6200895E0939503F0939603DB
:103B2C0060939703709398030895E0917503F09157
:103B3C00760360917703709178030895EAE0F0E0E2
:103B4C000E9490220895A0917503B0917603809104
:103B5C0077039091780308951ADC1ECCE0937103DF
:103B6C00F093720360937303709374030895F0E001
:103B7C00EA0FFB1FE0933303F0933403AEE30C9492
:103B8C0056190E945619A0E00C945619E091340372
:103B9C00AE2F0E945619A09133030C945619B0E025
:103BAC00E2E0F0E00E94A3220895EAE0E8AFE9AF7A
:103BBC00EAAF0895A0916D03B0916E0380916F03ED
:103BCC009091700308950E9450220E2EF3CFAA30CC
:103BDC00E0E0BE07E0E08E07E0E09E07089574DCAD
:103BEC00EAE0F0E060E070E008950E94CD22DF0191
:103BFC00CB01EAE0F0E060E070E00E94E72208957B
:103C0C00DF01EAE0F0E00E94D5220895A0911F03A5
:103C1C00BB27EAE0F0E00E94D5220895E4E6F0E04C
:103C2C0060E070E00895C6DFEAE0F0E060E070E08C
:103C3C000895A0E022FCA1E0EA2FEE0F08950E2ECD
:103C4C00A0E022FCA1E0EA2FEE0FEE0FE00DEE8FCC
:103C5C000895A0912D03B0912E030895E4E6F0E0B1
:103C6C000E949022DF01EAE0F0E00E94D222EDAF48
:103C7C000895DF01EAE0F0E00E94D2220895EAE024
:103C8C00F0E00E94D2220895BB27EAE0F0E00E9407
:103C9C00D5220895E89420F8CCCF0E94A822DF0109
:103CAC00CB01EAE0F0E060E070E00E94E3220895CE
:103CBC00F8DBEAE0F0E060E070E00895DF01CB01B2
:103CCC00E0E0F0E060E171EC0E9499210895DF01E1
:103CDC00CB01E0E0F0E066EC72EC0E9499210895D3
:103CEC00DF01CB01E0E0F0EC69E774EC0E94992174
:103CFC000895A0915903B0915A030895E0E1F7E2B9
:103D0C000E94A3227DCFE8EEF3E00E94A32278CF9D
:103D1C00E4E6F0E00E94A32273CFEAE0F0E00E9418
:103D2C00D522EFAF089533DBE4E65ACBA0915B03C9
:103D3C00B0915C030895EB81FC81F695E7950895AD
:103D4C000E94902296CFA0913B03B0913C03089522
:103D5C00E0912003E170EE0FE0580895E695E695AA
:103D6C00E170EE0FEE0F08950E2EA0E0F199A1E098
:103D7C00EA2FEE0FEE0FEE0F08950E0EA0E020FCD2
:103D8C00A1E0EA2FE295E07FE00D0895E52FF0E049
:103D9C00DE01D096AE0FBF1F08950E9405220E2E95
:103DAC00AA8108950E9405220E2AAA810895AF8146
:103DBC00B885C4CEE3E10E940522E0290895E62DE2
:103DCC00F0E0DE011D96AE0FBF1F0895A0916103B8
:103DDC00B091620380916303909164030895EC9118
:103DEC00F0E00E94FB21A8E0BCE481E090E00E949E
:103DFC00CD22ECCFE0936103F093620360936303F5
:103E0C00709364030895E2DF6CCCE985FA855CDB82
:103E1C00662777270E948B22EDCFA0916903B09182
:103E2C006A0380916B0390916C030895EDABF5DF01
:103E3C00EAE0F0E060E070E0D8CEEEABEEDFEAE076
:103E4C00F0E060E070E00E94E722EFAB08950DDC3B
:103E5C00F695E795D5CBEC8F32DAA436E0E0BE07C9
:103E6C0008952DDAE4E6F0E06BCF29DA67CE27DA95
:103E7C0006CFA0914903B0914A030895E9E3E9AF55
:103E8C00E0E5EAAFEEE3EBAF0895A0913103B0911A
:103E9C0032030895A0913F03B09140030895E1705F
:103EAC00E795E0E0E795AE2F0895E295EF70E69583
:103EBC00E170E295E07FEE0FEE0FEA2BAE2F089546
:103ECC00E295EF70E695E695E170E295E07FEE0FF6
:103EDC00EA2BAE2F0895E295E170E295E07FEA2B94
:103EEC00AE2F0895E170EE0FEE0FEE0FEA2BAE2F12
:103EFC000895E695E170EE0FEE0FEA2BAE2F0895C4
:103F0C00E695E695E170EE0FEA2BAE2F0895E69557
:103F1C00E695E695E170EA2B0895E695E170E29559
:103F2C00E07FEE0FEE0FEA2BAE2F0895E695E695A7
:103F3C00E170E295E07FEE0FEA2BAE2F0895E69547
:103F4C00E695E695E170E295E07FEA2BAE2FEE8DDB
:103F5C000895E695E695E695C5CFE295EF70E69562
:103F6C00E170EE0FEE0FEA2BAE2F0895E295EF7095
:103F7C00E695E695E170EE0FEA2BAE2F0895E295EB
:103F8C00EF70E6958CCFE295EF70E695E695089587
:103F9C00E170E295E07FEA2BAE2F0895E170E29597
:103FAC00E07FEE0FEE0FEA2BAE2F0895E695E17051
:103FBC00E295E07FEE0FEA2BAE2F0895E170EE0F45
:103FCC00EA2BAE2F0895E295EF70E695E1CF289895
:103FDC0085E28A95F1F751E008955E9885E28A951D
:103FEC00F1F7ECE0E51B089585E28A95F1F75E9A0E
:103FFC0085E28A95F1F708955D9A85E28A95F1F745
:10400C00289A84E191E00197F1F7E1CF109639F00D
:10401C008DEC9AE00197F1F7A8951197C9F70895DF
:10402C00552342F4503811F4E0FF04C03196691F57
:10403C00791F6BF050E8572711F45F93CFC05F3FA7
:10404C0031F0660F000C57956795752F08955F93A7
:10405C0000200AF0CFC0C8C050E8192E1522880FD6
:10406C00991F9527550F879550E8072E0522660F47
:10407C00771F7527550F67950895689401C0E894CC
:10408C005F93F2DF703818F07F3F08F4A7C056E159
:10409C00571BAAF4519558300EF4593030F0EFEF0D
:1040AC00FFEF6FEF7FE777F91AC077275523B9F049
:1040BC00EE0FFF1F661F771F5A95D1F710C0772799
:1040CC00583028F0EF2FF62F672F5850F9CF552383
:1040DC0031F076956795F795E7955A95D1F70020CD
:1040EC000AF45BD15F910895689401C0E89430970D
:1040FC0060407040B1F0002426F0772312F4009455
:10410C004CD1172E7EE1112032F07A95EE0FFF1F65
:10411C00661F111CF9CFEF2FF62F612D5F938ADFED
:10412C005F9108954F93AF01FD01DA01AB01BC0122
:10413C00CA01402D012C142E4F910895EA0FFB1F3C
:10414C00681F0895E095F0956095EF5FFF4F6F4FF6
:10415C0008955F9381DF903871F150E8152604C003
:10416C005F937ADF903839F1703821F1572F591B52
:10417C002BF112F4D7DFFACF583118F0AA27BB274E
:10418C008827583028F0AB2FB82F88275850F9CFF4
:10419C00552329F08695B795A7955A95D9F7502DA3
:1041AC00512572F0CBDF38F46795F795E795739549
:1041BC0013F420C0B7DF3EDF5F910895D8F7FBCF33
:1041CC00EA1BFB0B680B51F010F40094BBDF662369
:1041DC0092F3EE0FFF1F661F7A95CBF7EE27FF27A2
:1041EC00662777275F910895EFEFFFEF6FE77FEF7B
:1041FC005F910895EFEFFFEF6FE77FE75F91089511
:10420C005F932ADF703851F3903841F301240894FE
:10421C00791F23F41CF300203AF3ECCF0F921F9379
:10422C002F933F934F93112722279927689FA00123
:10423C008F9F302D410D591F6B9F300D411D591F04
:10424C008E9F27D0BF9F25D06A9F23D0BE9F1DD0A5
:10425C00AF9F1BD0AE9F110D291F391F491F591F2E
:10426C00E32FF42F652F522F4F913F912F911F91D8
:10427C000F9066232AF0550FEE1FFF1F661F02C01A
:10428C0073954BF2CDDE5F910895100D211D391FF2
:10429C0002C0200D311D491F591F08955F93DCDEAC
:1042AC00703821F411200AF49FCFA4CF903809F470
:1042BC0095CF01240894970B1BF4D4F30020F3CF73
:1042CC00792F1F932F933F934F931124112722275C
:1042DC0033274427552790E2AE17BF0786074107BF
:1042EC0030F0AE1BBF0B860B410B089401C08894B9
:1042FC00551F221F331F111CAA1FBB1F881F441FD1
:10430C009A9551F7F901612D4F913F912F911F9182
:10431C00662332F0550FEE1FFF1F661F7A9543F28E
:10432C007FDE5F91089599239AF0772342F09717D7
:10433C0048F029F4AE17BF07860720F031F09894A7
:10434C0088940895989408940895189488940895DE
:10435C007723C2F7971798F3A9F7EA17FB076807B3
:10436C0088F399F3ECCFDFDFE1E009F008F0EE27FA
:10437C000895D9DFE1E009F008F4EE270895EA0F7B
:10438C00FB1F681F791F0895AE1BBF0B860B970B85
:10439C000895F195E195F0400895F095609570952C
:1043AC00E195FF4F6F4F7F4F0895EE230E2EEA2FAE
:1043BC0019F0E6950A94E9F70895EE230E2EFD0107
:1043CC0021F0F695E7950A94E1F70895F695E795AF
:1043DC00F695E795F695E795F695E7950895FE2FF2
:1043EC00FF0FFF0B6F2F7F2F08956F2F660F660B3C
:1043FC00762F08958B2F880F880B982F0895EA1726
:10440C00E1E009F0EE270895EA17E1E009F4EE2760
:10441C000895AE17E1E00CF4EE270895AE17E1E035
:10442C000CF0EE270895EA17E1E00CF0EE27089562
:10443C00AE17E1E008F0EE270895EA17E1E008F086
:10444C00EE270895EA17FB07E1E009F0EE2708953F
:10445C00AE17BF07E1E008F4EE270895AE17BF07CB
:10446C00E1E008F0EE270895EA17FB07E1E008F019
:10447C00EE270895EA17FB0768077907E1E009F0D2
:10448C00EE270895AE17BF0786079707E1E00CF0FB
:10449C00EE270895EA17FB0768077907E1E00CF0AF
:1044AC00EE270895FA9FF02DEB9FF00DEA9FE02D7B
:1044BC00F10D08957A9F702D6B9F700DF89F700D04
:1044CC00E99F700D6A9F602D710DFB9F600D711D32
:1044DC00E89F600D711D8827FA9FF02D610D781FE4
:1044EC00EB9FF00D611D781FEA9FE02DF10D681F09
:1044FC00781F08956E2F6A9FF0016B9FF00D089541
:10450C0074D0D0DF0EF445DF08957DD0D3DF0EF4E8
:10451C0044DF08950024112490E1AA0FBB1F001C56
:10452C00111C0E1A1F0A18F40E0E1F1E01C0A160DA
:10453C009A9599F7FD01D001089557D0EBDF0EF451
:10454C0028DF08953F934F935F9300241124442751
:10455C00552730E2AA0FBB1F881F991F001C111C86
:10456C00441F551F0E1A1F0A460B570B28F40E0E2C
:10457C001F1E461F571F01C0A1603A9559F7FD0138
:10458C00BC01D001CA015F914F913F9108953BD07E
:10459C00D9DF0EF402DF0895BDDFFD010895E89424
:1045AC00B7FF04C0A095B09511966894F7FDF1DEA5
:1045BC00B1DFFD010EF4EDDE0895C4DFFD01BC0199
:1045CC000895E89497FF09C0A095B09580959095B3
:1045DC00AF5FBF4F8F4F9F4F689477FDDEDEB2DF2A
:1045EC00FD01BC010EF4D9DE0895E894F7FF02C07A
:1045FC00D0DE6894B7FF06C0A095B095119600F870
:10460C00039400FA0895E89477FF02C0C6DE68941C
:10461C0097FF0BC00024A095B095809590951196AE
:10462C00801D901D00F8039400FA0895ED93FD93FE
:10463C006D937C930895689401C0E89401D057DD84
:10464C00182E862F612D192E972F712D1B2EBF2FF3
:10465C00F12D1A2EAE2FE12D0895129602D0BF0126
:10466C001297119602D0FE2F1197F999FECFFF9356
:10467C00FFB7F894A1BDB2BDF89AE0B5FFBFFF91AA
:10468C00089507D012960F01FB0103D0F001129789
:10469C00089507D01196EF93EF2F03D0EF91119758
:1046AC000895F99B02C0A895FCCF9FB7F894A1BDC3
:1046BC00B2BDF89A80B5E81719F0E0BDFA9AF99AEC
:1046CC009FBF089500240E160F06060607060895D0
:1046DC0000240A160B06089500240A160B06080679
:1046EC0009060895EA17FB07680779070895AE17BE
:1046FC00BF07860797070895E894EE2309F068949E
:10470C000895AC0FBD1F05900D928A95E1F70895A1
:00000001FF
